:040000008A15002835
:10000800FF00030E830103179D000A089C008A0164
:1000180070080313C1007108C0000408C2008316E9
:100028008C1E812883128C1E8128981C2B2818125C
:100038000000181683165608013EF0000030031819
:10004800013E5707F1007008D6007108D7008312E7
:10005800181D3E2898130000981783165608013E6D
:10006800F00000300318013E5707F1007008D60071
:100078007108D70083121A08031790001008031399
:100088009900031710080D3A031D642883160313FB
:100098006E178C12831203171108203E840080010A
:1000A800110883160313DA00831203171208831644
:1000B8000313DB0083120317910192019001812839
:1000C8001108203E840010088000110883160313CD
:1000D800DA0083120317120883160313DB00831256
:1000E80003171108013EF00000300318013E120703
:1000F800F1007008910071089200031383124108FF
:10010800F0004008F1004208840003171C088A0028
:0A0118001D0E8300FF0E7F0E09008C
:0E012200213083120313FD00FD0B9528080009
:06013000000000000800C1
:100136000F3083120313FC004730FD00FD0BA1288E
:0A014600FC0BA128000000000800D7
:0E015000831203171B088A001A088200080099
:10015E0083120313F801F9011030FC00710DF80D34
:10016E00F90D7408F8027508031C750FF9020318CF
:10017E00C7287408F80775080318750FF9070310D8
:0A018E00F00DF10DFC0BB528080080
:10019800831603139818D2280000CC28831203175B
:0801A8002A0803139900080066
:1001B000710DF80DF90D7408F8027508031C750F20
:1001C000F902F00DF10D0F30FC00710DF80DF90D75
:1001D0007408701CF128F8027508031C750FF902E9
:1001E000F628F80775080318750FF907F00DF10DDB
:1001F000FC0BE528701802297408F8077508031825
:08020000750FF907000008006A
:1002080083120317AA1B0A2986110B2986152A1B94
:100218000F29061110290615AA1A1429861015295E
:1002280086142A1A192906101A29061416181F29BD
:10023800031385152129031385118514982085102A
:100248000317AA19292986112A2986152A192E2958
:1002580006112F290615AA18332986103429861461
:100268002A18382906103929061416183E290313A6
:1002780085154029031385118514982085100317C7
:0C028800161C48299B20492991200800E1
:10029400831203137408003A031D59297508003AA0
:1002A400031D5929FF30F0007F30F100B229831279
:1002B4000313FD01F901F8017108700403190034F6
:1002C40071087506FA00FA1BFD09FB01F51F6F2979
:1002D400F409F509F40A0319F50AF11F7629F0095E
:1002E400F109F00A0319F10A71087504FA00FA1BFE
:1002F4008B29D8207B189E29FD1F0034F009F109B1
:10030400F00A0319F10AF809F909F80A0319F90AB4
:100314000034F51F9A29F11B96297108F900700819
:10032400F800F101F0017E29F101F001F00A003436
:10033400F109F009FB0A7B29F80A0319F90A740880
:100344007802031D7E2975087902031D7E29F901AF
:10035400F801F00A0319F10AF11F7E290000FF34A5
:0203640008008F
:100366000D3083120317AA00CC200A300317AA0007
:04037600CC2008008F
:10037A0083120313F8010830FC00700DF80D74089D
:10038A00F8020318CA29F8070310F00DFC0BC2295A
:02039A00080059
:10039C0083120317A801053028020318DC2928084A
:1003AC002707840020308000A80AD12928082707B5
:1003BC0084008001A80328082707A9000A30F4004C
:1003CC00F5012508F0002608F100AF207808F000B0
:1003DC007908F1003030F007031729088400700801
:1003EC0080000A30F400F5012508F0002608F10021
:1003FC00AF2070080317A5007108A6000030710625
:10040C00031D0A2A00307006031D0D2A0F2AA803AB
:04041C00E1290800CA
:100420008312031725089A0026089B00A8208A112A
:100430000A12F000700803192B2A25089A002608D2
:100440009B00A8208A110A12AA00CC200317A50A33
:080450000319A60A102A080096
:100458008312031716102508AA000421031716147F
:0204680008008A
:10046A00831203172708F000A703700803195D2AEF
:10047A00250884000008003A03194E2A2608840039
:10048A000008F1002508840000087106031D4E2AA1
:10049A005A2A250884000008F0002608840000086B
:1004AA00F002F101031CF1035F2AA50AA60A352A04
:0604BA00F001F101080051
:1004C000831203172508F2007208F000F20A700880
:1004D0008400000803196D2A642A25087202F000BE
:0C04E0000130F002F101031CF1030800E0
:1004EC0083120317A701250884000008A60026081C
:1004FC00003A03198C2A2608AA00CC200317A70A55
:0E050C002708250784000008A6007D2A0800A5
:10051A00831203172508840000082606031D982A5B
:10052A002508F000A32A2508F000A50A700884000F
:0E053A000008F0007008031D8D2AF001080073
:1005480083120317A101A201A301A4011E08073CFD
:100558000318B12AF001F101472BC73003139F0597
:1005680003171E08F000F00D7010F00D7010F00D5C
:100578007010700803139F040830FC00C930FD0098
:10058800FD0BC42AFC0BC42A0000000003179F01BE
:10059800A00180302006F00080307002031DD62AAA
:1005A80010301F020318302B03139F1400009F1CE8
:1005B800DE2ADB2A1E080317A400A30183160313EF
:1005C8001E0883120317A3070318A40A2308A10708
:1005D80024080318013EA207831603136E1E202B5E
:1005E8000830F4000030F500831203171F08F000EC
:1005F8002008F1004A217808F0007908F10000305D
:100608007106031D092B00307006031D122BB32140
:10061800D5300317A5000B30A600102203172308B6
:10062800A5002408A600DC30A700CE21DC30A500F8
:1006380076220930AA00CC200330FC009730FD0058
:100648008312FD0B242BFC0B242B00000000031746
:100658009F0A0319A00ACD2A21080313E7000317EC
:1006680022080313E800E80CE70CE813E80CE70C91
:10067800E813E80CE70CE813E80CE70CE813670844
:08068800F0006808F100080011
:1006900083120317A001033020020318562B2008F1
:1006A0001F07840020308000A00A4B2B20081F0762
:1006B00084008001A00320081F07A1000A30F40075
:1006C0001E08F000BD217808F0003030F007031755
:1006D00021088400700880000A30F4001E08F00031
:1006E000BD21700803179E007008003A031D792B86
:0806F0007B2BA0035B2B08002B
:1006F80083120313FB01FA01F9018030F800F10CB1
:10070800F00C031C902B7408F90775080318750F73
:10071800FA070318FB0A0310F01F982B7408FA074E
:1007280075080318750FFB07FB0CFA0CF90CF80C8D
:10073800031C832B7B08F3007A08F2007908F10088
:060748007808F000080033
:10074E00831203171E08003A0319D12B1E088400CA
:10075E0000080319D12B1F08A50060227008A700FE
:10076E001E08A5001F08A600352200307106031DC5
:10077E00C22B00307006031DC72B1E08F000D22BB3
:10078E001E0AA5001F0884000008A6008D2270080E
:08079E009E00A72BF0010800EA
:1007A6000B3083120313FB002630FC005D30FD0086
:1007B600FD0BDB2BFC0BDB2BFB0BDB2B000000000C
:0207C600080029
:1007C80083160313DA01DB0180305B06F00080300A
:1007D8007002031DF12B20305A020318042C5A080A
:1007E800203E840080015A08013EF00000300318C2
:1007F800013E5B07F1007008DA007108DB00E82BA6
:10080800DA01DB01831203179101920183160313A6
:100818006E1383121A0803179000900183160313AE
:06082800EF018C16080030
:10082E00831203179F011F081E0784000008031977
:10083E00282C1F081E0784000008A5002C229F0AE2
:04084E001A2C080058
:10085200A8208A110A128000840A9A0A03199B0AA4
:08086200F003031D292C08001E
:10086A0083160313981690308312980083168717FD
:10087A00071383128C1E442C1A08F0003E2C080021
:10088A00831203171E08F2007208F100F20A1F0809
:10089A00F0009F0A700884000008F00071088400C4
:1008AA007008800071088400000803195D2C492C27
:0608BA001E08F00008001A
:1008C0008130831203139F008E3083169F0008002F
:1008D00083160313851085110610861006118611E4
:1008E00083128510851186110611861006109B2033
:1008F0009B209B20861406148514982085109B202D
:100900008514982085109B208514982085109B20A5
:1009100006108514982085109B208514982085103A
:10092000861086158514982085109B208611061444
:1009300085149820851006108514982085109B201A
:1009400085149820851006148514982085109B2006
:100950000610851498208510861506158614061431
:0E0960008514982085109B200317161408009C
:10096E00831203137008F100F0010830FC007108C7
:10097E00F40C0318C62CFC0BBF2CF1010034031031
:10098E00CB2CF40C0318F107F10CF00CFC0BC82C5B
:02099E0008004F
:10100000DE237130831603138F00F1308500031740
:101010008801013088008901831287138813FF300B
:10102000831603138600FF3087008E309F00BB308D
:1010300087008801F030860083128501831607102F
:10104000851605160813831208138316DA01DB01CF
:1010500080305B06F00080307002031D31282030A4
:101060005A02031844285A08203E840080015A0876
:10107000013EF00000300318013E5B07F1007008EC
:10108000DA007108DB002828DA01DB01831203177C
:1010900091019201831603136E132030EF00193073
:1010A000990018158A1135248A158A11B3218A15D9
:1010B00087300317A5000B30A6008A1110228A156D
:1010C00083160313D801D90100305902031D6A2881
:1010D0000730580203189028F0018312081BF00A09
:1010E0000130F007F1010318F10A0230F000831615
:1010F0005808F4008A11B7248A157008433E84000A
:1011000000080317A500840A0008A6008A1110220F
:101110008A15031308138316D80A0319D90A6428F9
:101120008A11B3218A150E300317A5000730A600D7
:101130008A1110228A15031307108316D601D701CE
:101140000C3083120317AA008A11CC208A150630AE
:10115000FB001330FC00AD30FD00FD0BAD28FC0B97
:10116000AD28FB0BAD2800000000CA300317A50016
:101170000B30A6008A1110228A158A1160248A1564
:10118000A73083120317A5000B30A6008A11102286
:101190008A159C30A5000730A6008A1110228A15F6
:1011A0000313880188168A1168248A158030AA00E2
:1011B0008A1104218A15DC3003179E00A0309F009D
:1011C0008A1145248A15DC309E008A1117248A155D
:1011D0001530FB004B30FC00BE30FD00FD0BEE284F
:1011E000FC0BEE28FB0BEE280000C030AA008A1191
:1011F00004218A15DC3003179E0053309F008A11AA
:1012000045248A15DC309E008A1117248A150B307C
:10121000FB002630FC005D30FD00FD0B0D29FC0BB2
:101220000D29FB0B0D2900000000831603138C1001
:1012300083120817831607150C30831297000C30A1
:101240009D00121792161216921592141210FF306A
:10125000831692007F308312031793001308031341
:10126000950008171215081383160711DA01DB0120
:101270006E13831203179101920183160313DA018F
:10128000DB01831218160B1783168C168B17EE13BF
:10129000D03083120317A5000430A6008A11102253
:1012A0008A158A11B3218A1583166E168A11E423D2
:1012B0008A158A11D3238A1583166E1FA82AF73040
:1012C00083120317A5000730A6008A1110228A1581
:1012D0002030A5008A1176228A1520309E00C23067
:1012E0009F008A11A7238A15700883160313EF0045
:1012F0006F08003C0318152A08306F07840080012E
:1013000005306F07840030300002F000F101031C4B
:10131000F1036430F4000030F5008A117C238A1553
:10132000700803179800710899000630831603139C
:101330006F07840030300002F000F101031CF1035C
:101340000A30F4000030F5008A117C238A157008F9
:101350000317980771080318013E99070730831691
:1013600003136F07840030300002F000F101031C0A
:10137000F103700883120317980771080318013EE0
:1013800099071808A5001908A600DC30A7008A11E3
:10139000CE218A15DC30A5008A1176228A15093003
:1013A000AA008A11CC208A1503171908003C031DD6
:1013B000DB291808003C0318FB2900301902031D23
:1013C000E329C83018020318FB29FF3018059300E1
:1013D0000313121103171308031395001215BF30DE
:1013E0000317A5000B30A6008A1110228A15831658
:1013F0000313EE13152A831203171808A500190802
:10140000A600DC30A7008A11CE218A159A30A500EB
:101410000B30A6008A1110228A15DC30A5008A1133
:1014200076228A158A11B3218A1583122030031778
:101430009E0069309F008A11A7238A1570088316C1
:101440000313EF006F08003C0318302AEE17253015
:1014500083120317A5000B30A6008A1110228A15EB
:101460008312031720309E00CE309F008A11A723DD
:101470008A15700883160313EF006F08003C0318E9
:101480004B2AEE137C3083120317A5000730A60009
:101490008A1110228A158312031720309E00CB3048
:1014A0009F008A11A7238A15700883160313EF0083
:1014B0006F08003C03186A2A83121211593003176F
:1014C000A5000B30A6008A1110228A150313921072
:1014D000121012158312203003179E00C8309F008F
:1014E0008A11A7238A15700883160313EF006F086B
:1014F000003C0318892A831212110A300317A50031
:101500000B30A6008A1110228A15031392141210B0
:1015100012158312203003179E0064309F008A1139
:10152000A7238A15700883160313EF006F08003C89
:101530000318A82A831212113F300317A5000B309D
:10154000A6008A1110228A15031392101214121584
:101550008316EE1FC62A8A11B3218A1503171408B1
:10156000F0001508F100F10CF00CF113711BF117EC
:10157000F10CF00CF113711BF117700893000313B9
:1015800012110317130803139500121583128030EC
:101590000317AA008A1104218A15DC3003179E0064
:1015A000B1309F008A1145248A1513089E00E93046
:1015B0009F008A1148238A1583160313EC01DC303F
:1015C000831203179E008A1117248A150313081724
:1015D000DC300317A5008A1176228A158A11B321FF
:1015E0008A1508130317970117089E008A11A42271
:1015F0008A1583120313700803179400710895006D
:0A1600008A11B3218A155629042B24
:1017BC0043308400213083120313F0005B30031795
:1017CC009A0007309B008A1129248A15A0308400C6
:1017DC0022308312F000393003179A0007309B0037
:1017EC008A1129248A15643084000C308312F0008D
:1017FC00B33003179A000B309B008A1129248A15E9
:10180C00C230840014308312F000733003179A0036
:0C181C000B309B008A1129248A1508005B
:1009A0002034543465347334743420345034573420
:1009B0004D342034203461347434203446344F3480
:1009C000533443343D34323430344D3448347A3443
:1009D0002034203450346F34733474342D347334F1
:1009E000633461346C346534723420344E346F3483
:1009F0006E3420345534743469346C34693473344F
:100A0000E934213420345034523432343D343234D9
:100A1000353435340D340A3420345034723465346E
:100A20007334633461346C3465347234203420346C
:100A30003A342034203461347634653463342034DD
:100A400031342F3431343634203420344634723447
:100A5000653471343D342034343439343034203406
:100A600048347A3420340D340A3420344334683422
:100A70006F346934783420345034723465347334CC
:100A8000633461346C346534723420343A34203445
:100A90004834493447344834203420344D344534C4
:100AA0004434493455344D34203420344C344F349C
:100AB000573420340D340A342034443475347434BB
:100AC00079345F344334643465345F344D346F3487
:100AD00064346534203476346934613420344B34E2
:100AE0006534793462346F34613472346434203460
:100AF000203444347534743479343D347834783463
:080B000078340D340A3400348E
:100B0800203445344534503452344F344D34203435
:100B18003A3420343134363446343834383437347F
:100B28005F3449345234443441345F34643461347A
:100B380062346F346134723464345F3454346534ED
:100B48007334743473345F346D3469346E34693497
:100B58006D3461345F3446347234653471345F34D3
:100B6800503457344D345F347734693474346834CE
:100B78005F3446346F34733463345F3438344D34FF
:100B880068347A345F3432343034323430345F3459
:100B980045344534503452344F344D342E3469344E
:0C0BA8006834653478340D340A340034AD
:100BB400203453346F3475347234633465342034E0
:100BC4003A3420345F3431343634463438343834AB
:100BD40037345F34493472346434613462346F348A
:100BE4006134723464345F3454346534733474342B
:100BF40073345F34503457344D345F346134743457
:100C04005F3438344D3468347A345F3432343034B9
:100C1400323430345F3431343034303434342E347C
:100C240063345F3432343034323430345F3431340A
:100C34003034303434342E3463340D340A340034D4
:100C44002034503472346F346A3465346334743409
:100C540020343A3420343134363446343834383459
:100C640037345F3449345234443441345F34623469
:100C74006F346134723464345F345434653473349F
:100C8400743473345F34503457344D345F347734B0
:100C94006934743468345F3446346F347334633481
:100CA4005F3438344D3468347A345F343234303419
:100CB400323430342E346D346334703470346934E7
:060CC4000D340A34003477
:100CCA0020344434693472346534633474346F3490
:100CDA007234793420343A34203443343A345C342C
:100CEA005F344D3469346B3472346F3443345C345A
:100CFA005F344D3465347334503472346F346A342B
:100D0A006534743473345F344D3469346B347234FB
:100D1A006F3443345C345F343134363446343834D7
:100D2A00373437345F3449345234443441345F34CD
:100D3A0042346F346134723464340D340A3400340A
:100D4A0020344D3469346B3472346F344334203474
:100D5A0037342E34363430342E342034263420348A
:100D6A004D346934633472346F34633468346934AB
:100D7A007034203449345234443441342034623497
:100D8A006F34613472346434203431343634463446
:100D9A0038343834373420342834653478342034BD
:100DAA0031343634463438343734373429340D3410
:040DBA000A340034C3
:100DBE00203463346F346E347334693467346E3474
:100DCE0065342034503457344D34203476346934FD
:100DDE00613420344B346534793462346F34613489
:100DEE007234643420346F347534203470346F347C
:100DFE007434613472342034733475347234203464
:0E0E0E0045344134303420340D340A3400347D
:100E1C00203452346534733465347434203464347F
:100E2C00753420344D344334503432343134353409
:100E3C0030342C34203470346F34753472342034A4
:100E4C007534743469346C34693473346534723485
:100E5C0020345234583420345534413452345434C0
:060E6C000D340A340034CD
:100E72003134363446343834383437342034493413
:100E820052344434413462346F34613472346434E1
:020E920000342A
:100E940044347534743479342034563461346C34C5
:100EA400753465343D3420342034203420342034E7
:020EB400003408
:100EB600A53406346534063422340634DA3405346F
:100EC600DA34073484340534BB340734DF3406346B
:100ED600503457344D3420346F3475347434703490
:100EE6007534743420346F346E34523443343234AF
:020EF6000034C6
:100EF8000D340A34203444347534743479345F340E
:100F08004334643465345F344D346F346434653449
:100F1800203476346934613420344B346534793480
:100F280062346F346134723464340D340A340034FA
:100F3800203450346F3477346534723420344F346D
:100F48006E3420342834523444343534293420342F
:100F580061346E346434203449346E346934743402
:0E0F680020344C34433444340D340A34003405
:100F760020345434453453345434203450345734A4
:100F86004D3420343A34203473346F34723474342C
:100F960069346534203473347534723420345234F1
:0E0FA60043343234203420340D340A34003405
:100FB400203446346F347334633420343D34203465
:100FC40049346E347434653472346E3461346C3440
:100FD400203446344F3453344334203438344D347D
:0A0FE40048347A340D340A34003426
:100FEE000D340A3452346534E734753420343A34CF
:020FFE000034BD
:101614000D340A3420347334653474342034503433
:10162400723465347334633461346C3465347234C5
:101634002034E034203431342F34313436342034FF
:061644000D340A340034ED
:10164A000D340A34203444347534743479345F34B4
:10165A004334643465345F344D346F3464346534F0
:10166A0020346634283445344134303429340D3436
:04167A000A340034FA
:10167E000D340A34203473346534743420345034C9
:10168E00723465347334633461346C34653472345B
:10169E002034E034203431342F34343420340D34BB
:0416AE000A340034C6
:1016B2000D340A3420347334653474342034503495
:1016C200723465347334633461346C346534723427
:1016D2002034E034203431342F34313420340D348A
:0416E2000A34003492
:0C16E60044347534743479343D340034DD
:0616F2004C344F340034BB
:0616F800483449340034BF
:1016FE0041344E3441345F344F3446344634003432
:10170E002034503472346534733465346E3474342A
:10171E006134743469346F346E3420343A34203486
:06172E000D340A34003402
:101734004234613464342034763461346C34753426
:0A174400653420343A3420340034B8
:10174E00203449346E346934743420344C34433488
:08175E0044340D340A34003458
:061766004D34453400344F
:04176C000034003411
:0E17700041344E3441345F344F344E34003433
:10177E0020342D343E3420344F344B3420340D3449
:06178E000A34203400348F
:10179400413444344334203449346E346934743429
:0617A4000D340A3400348C
:1017AA00203445344134303420343D343E342034FE
:0217BA000034F9
:04400E00F42C000787
:020000040000FA
:1042000031003600460038003700370020006F00CC
:104210006E0020004900520044004100200042008E
:104220006F0061007200640020002B0020004C0031
:104230004300440020002B005100320030004D00AC
:1042400048007A000D000A000000FF00FF00FF0098
:10425000FF00FF00FF00FF00FF00FF00FF00FF0066
:10426000FF00FF00FF00FF00FF00FF00FF00FF0056
:10427000FF00FF00FF00FF00FF00FF00FF00FF0046
:10428000FF00FF00FF00FF00FF00FF00FF00FF0036
:10429000FF00FF00FF00FF00FF00FF00FF00FF0026
:1042A000FF00FF00FF00FF00FF00FF00FF00FF0016
:1042B000FF00FF00FF00FF00FF00FF00FF00FF0006
:1042C000FF00FF00FF00FF00FF00FF00FF00FF00F6
:1042D000FF00FF00FF00FF00FF00FF00FF00FF00E6
:1042E000FF00FF00FF00FF00FF00FF00FF00FF00D6
:1042F000FF00FF00FF00FF00FF00FF00FF00FF00C6
:10430000FF00FF00FF00FF00FF00FF00FF00FF00B5
:10431000FF00FF00FF00FF00FF00FF00FF00FF00A5
:10432000FF00FF00FF00FF00FF00FF00FF00FF0095
:10433000FF00FF00FF00FF00FF00FF00FF00FF0085
:10434000FF00FF00FF00FF00FF00FF00FF00FF0075
:10435000FF00FF00FF00FF00FF00FF00FF00FF0065
:10436000FF00FF00FF00FF00FF00FF00FF00FF0055
:10437000FF00FF00FF00FF00FF00FF00FF00FF0045
:10438000FF00FF00FF00FF00FF00FF00FF00FF0035
:10439000FF00FF00FF00FF00FF00FF00FF00FF0025
:1043A000FF00FF00FF00FF00FF00FF00FF00FF0015
:1043B000FF00FF00FF00FF00FF00FF00FF00FF0005
:1043C0007000610075006C0066006A0075006A008C
:1043D0006F00400066007200650065002E006600F8
:1043E00072002000310035002D00300031002D001A
:1043F0003200300031003400FF00FF00FF00FF00FA
:00000001FF
